:020000040800F2
:1000000000040020E5010008DD0E0008E10E0008F4
:10001000350F0008E10E0008090F0008E70100088D
:10002000E7010008E7010008E7010008BD27000814
:10003000E7010008E7010008E7010008E701000800
:10004000E7010008E7010008E7010008E7010008F0
:10005000E7010008E70100080D39000839390008F8
:100060006539000891390008BD390008E70100082A
:10007000E7010008E7010008E7010008E7010008C0
:10008000E7010008E7010008E7010008E7010008B0
:10009000E7010008E7010008E7010008E939000866
:1000A000E7010008E7010008E7010008E701000890
:1000B00029370008E7010008E7010008E701000808
:1000C000E7010008E7010008E7010008E701000870
:1000D000E7010008E5100008F9100008E701000832
:1000E000513A0008E7010008E7010008E7010008AD
:1000F000E7010008E7010008E7010008E701000840
:10010000E7010008E7010008E7010008E70100082F
:10011000E70100080D110008E7010008E7010008E9
:10012000E7010008E7010008E7010008E70100080F
:10013000E7010008E7010008E7010008E7010008FF
:10014000E7010008E7010008E7010008A92E000800
:10015000E7010008E7010008E7010008E7010008DF
:10016000E7010008E7010008E7010008E7010008CF
:10017000E7010008E7010008E7010008E7010008BF
:10018000E7010008E7010008E7010008E7010008AF
:10019000E7010008E7010008E7010008E70100089F
:1001A000E7010008E7010008E7010008E70100088F
:1001B000E7010008E7010008E7010008E70100087F
:1001C000E7010008E7010008E7010008E70100086F
:1001D000E7010008E7010008E7010008E70100085F
:1001E000BD0E000802E000F000F8FEE772B63948E4
:1001F00080F30888384880F3098838484EF608515B
:10020000CEF20001086040F20000CCF200004EF691
:100210003471CEF200010860BFF34F8FBFF36F8FD0
:1002200040F20000C0F2F0004EF68851CEF200011C
:100230000860BFF34F8FBFF36F8F4FF00000E1EE08
:10024000100A4EF63C71CEF200010860062080F3E1
:100250001488BFF36F8F02F0EFFA03F0FBF94FF051
:1002600055301F491B4A91423CBF41F8040BFAE745
:100270001C49194A91423CBF41F8040BFAE71A495C
:100280001A4A1B4B9A423EBF51F8040B42F8040B2A
:10029000F8E700201749184A91423CBF41F8040B87
:1002A000FAE702F0CDFA03F031FA144C144DAC42E7
:1002B00003DA54F8041B8847F9E700F03FF8114CC3
:1002C000114DAC4203DA54F8041B8847F9E702F0F9
:1002D000B5BA00000004002000240020000000083F
:1002E0000000002000040020B83E00080024002088
:1002F0002824002028240020783D0020E001000868
:10030000E4010008E4010008E40100082DE9F04FD1
:100310002DED108AC1F80CD0C3689D46BDEC108A43
:10032000BDE8F08F002383F311882846A047002002
:1003300001F0CAFE01F07AFE00DFFEE71A4B6FF013
:10034000780270B500241A700F225C709C70DC700B
:100350001C715C719C71DC711C725C729A72DC7233
:1003600002F0FEF9064602F023FA054650B90F4B9B
:100370009E4217D001339E4241F2883412BF054697
:1003800000240125002002F0F5F90DB100F0B4F8C9
:1003900000F036FD00F018FC204600F00BF900F0EC
:1003A000ABF8F9E70446EDE728240020010007B088
:1003B00008B500F087FBA0F120035842584108BD62
:1003C00007B5054B02211B88ADF8043001A800F0E9
:1003D000E5FB03B05DF804FB383B0008064991F8E3
:1003E000243033B100230822086A81F8243000F059
:1003F0000DBC0120704700BF482400202DE9F84FB4
:10040000234C94F824300546884617468BBB2E466D
:10041000DFF87C90002F38D094F824A0BAF1000FB8
:1004200005D12022FF214846266200F0D7FCCAF100
:100430000805BD4228BF3D465FFA85FBAD00414639
:100440002A4604EB8A0000F09FFC94F82430A7EBC6
:100450000B079B445FFA8BFBBBF1080F2E44A844AB
:10046000FFB284F824B0D5D1FFF7B8FF0028D1D16E
:1004700008E0266A06EB8306B042C9D0FFF7AEFF5C
:100480000028C4D10020BDE8F88F0120BDE8F88F16
:100490004824002010B5202383F311881248C36834
:1004A0000BB101F097FE0023104A0F484FF47A7108
:1004B00001F054FE002383F311880D4C236813B11F
:1004C0002368013B2360636813B16368013B636089
:1004D000084B1B7833B9636823B9022000F04AFC4B
:1004E0003223636010BD00BF34240020950400084F
:1004F000782500207024002010B5254B254953F89D
:10050000042F013200D110BD8B42F8D1224C234B75
:1005100022689A423AD9224B9B6803F1006303F5A3
:1005200080339A4232D2002000F068FB1D4B02203B
:10053000187000F015FC1C4B1A6C00221A64196E1E
:100540001A66196E596C5A64596E5A665A6E5A690F
:1005500042F080025A615A6922F080025A615A6957
:100560001A6942F000521A611A6922F000521A61A7
:100570001B6972B60D4A0E4B13601B68226820215E
:1005800081F311889D4683F30888104710BD00BF92
:10059000FCFF00081C00010804000108FFFF000820
:1005A00028240020702400200038024008ED00E0DC
:1005B000000001082DE9F04F99B0B34C01902022C2
:1005C000FF2110A8A66800F009FCB04A1378A346E2
:1005D000A3B9AF480121C3601170202383F31188B0
:1005E000C3680BB101F0F6FD0023AA4AA8484FF4F6
:1005F0007A7101F0B3FD002383F31188019B13B1DD
:10060000A54B019A1A60A54AA349019F02920023B3
:1006100013704B6099461C461D469846012000F019
:100620009FFB002F00F012829B4B1B68002B40F0B9
:100630000D8219B0BDE8F08F0220FFF7B9FE002847
:1006400040F0FB81019BB9F1000F08BF1F46944B9E
:100650001B88ADF82C3002210BA800F09FFADDE7D3
:100660004FF47A7000F02EFA031E0393EADB0220A7
:10067000FFF79EFE82460028E4D0039B581E042804
:1006800000F2DD81DFE800F0030E1114170018A856
:10069000052340F8343D042100F080FA54464FF021
:1006A000000856E004217848F6E704217D48F3E786
:1006B00004217D48F0E71C24204600F0A1FA043410
:1006C0000B9004210BA800F069FA2C2CF4D1E5E77B
:1006D000002DB7D0002CB5D00220FFF769FE0546EB
:1006E000002800F0AF8101206C4C00F087FA022056
:1006F000207000F035FB4FF000095FFA89FA504690
:1007000000F08CFA074658B1504600F097FA09F10C
:1007100001090028F1D12C46A9460027634B97E731
:1007200001230220237000F011FB3E46DBF8083065
:100730009E4206D2304600F063FA0130EBD1043617
:10074000F4E7029B00261E70534BA9465E602C46C0
:10075000374600F04BFB15B1002C18BF0027FFF700
:100760002FFE5BE7002D3FF46DAF002C3FF46AAF26
:10077000029B0220187000F0F3FA322000F0A2F978
:10078000B0F1000AC0F25E811AF0030540F05A8110
:10079000DBF8082006EB0A03934200F25381BAF516
:1007A000807F00F24F8155450DDA4FF47A7000F0EA
:1007B00089F90490049B002BC0F244813C4A049BBD
:1007C000AB540135EFE7C820FFF7F2FD05460028DE
:1007D00000F038811F2E11D8C6F12004544528BFDF
:1007E000544610AB26F0030022463149184400F06D
:1007F000CBFA2246FF212E4800F0F0FA4FEAAA0A6F
:100800005FFA8AF22A493046FFF7F8FD04460028CD
:1008100000F01A8106EB8A0605469AE70220FFF7E8
:10082000C7FD00283FF40EAFFFF7D8FD00283FF4C6
:1008300009AF4FF0000A5346DBF8082092451CD25E
:10084000BAF11F0F12D8109A01320FD02AF003020A
:1008500018A90A4452F8202C0B92184604220BA91E
:1008600000F07CFB0AF1040A0346E5E750460393D7
:1008700000F0C6F9039B0B90EFE718A8042140F89D
:100880004C3D00F08BF964E72824002074250020FB
:1008900034240020950400087825002070240020CE
:1008A0003A3B00082C240020302400203C3B000868
:1008B0007424002018A8002340F8343D642100F07F
:1008C00039F900287FF4BEAE0220FFF771FD002841
:1008D0003FF4B8AE0B9800F0C3F918AB43F8480DDD
:1008E00004211846CDE718A8002340F8343D6421C0
:1008F00000F020F900287FF4A5AE0220FFF758FD94
:1009000000283FF49FAE0B9800F0B8F918AB43F8FD
:10091000440DE5E70220FFF74BFD00283FF492AEBF
:1009200000F0B2F918AB43F8400DD9E70220FFF709
:100930003FFD00283FF486AE0BA9142000F0AAF971
:10094000824618A8042140F83CAD00F027F9514632
:100950000BA896E7322000F0B5F8B0F1000AFFF6D8
:1009600071AE1AF0030F7FF46DAEDBF808200AEBCE
:10097000080393423FF666AE0220FFF719FD0028F8
:100980003FF460AE2AF0030AC244D0453FF4E1AE22
:10099000404600F035F904210A900AA800F0FEF85C
:1009A00008F10408F1E74FF47A70FFF701FD002821
:1009B0003FF448AEFFF712FD00283FF4AFAE109BA6
:1009C00001330CD0082210A90020FFF717FD0028E2
:1009D0003FF4A4AE2022FF2110A800F0FFF9FFF79A
:1009E000EFFC374801F076FB23E6002D3FF42AAEFA
:1009F000002C3FF427AE18A8002340F8343D6421B2
:100A000000F098F8824600287FF41CAE0220FFF721
:100A1000CFFC00283FF416AE0390FFF7D1FC41F263
:100A2000883001F057FB0B9800F028FA00F0DEF94F
:100A3000039B57461C461D46F0E5054689E64FF0E8
:100A40000008FFE52546FDE52C4667E6002000F09E
:100A500039F80490049B002BFFF6E3AD012000F071
:100A600075F9049B213B122B3FF6D8AD01A252F839
:100A700023F000BF3906000861060008D10600080F
:100A80001D0600081D0600081D0600086507000871
:100A9000550900081D080008B5080008E708000807
:100AA000150900081D0600082D0900081D0600088C
:100AB000A7090008530700081D060008EB090008F5
:100AC000A08601002DE9F34702AE00244FF47A75A9
:100AD00006F8014D144FDFF85880454397F9003070
:100AE0005A1C5FFA84F901D0A34212D158F82400AD
:100AF00003680122D3F820A031462B46D0470128B5
:100B000007D10A4B9DF8070083F8009002B0BDE8BA
:100B1000F0870134042CE1D14FF4FA7001F0DAFAD5
:100B20004FF0FF30F2E700BF00240020982500209E
:100B30007C3B00082DE9F0474FF47A75144FDFF83D
:100B4000588006464D43002497F900305A1C5FFA3E
:100B500084F901D0A34210D158F82400036804227C
:100B6000D3F820A031462B46D047042805D1094BA5
:100B700083F800900020BDE8F0870134042CE3D115
:100B80004FF4FA7001F0A6FA4FF0FF30BDE8F0879D
:100B900000240020982500207C3B000830B4074B3F
:100BA0001A78074B53F822402368DD69054B0A4643
:100BB000AC460146204630BC604700BF9825002067
:100BC0007C3B0008A086010070B501F0CDFC094C0B
:100BD000094E2070002530682378834208D901F03F
:100BE000BDFC336805440133B5F5803F3360F2D373
:100BF00070BD00BF992500208025002001F062BD56
:100C000000F1006000F580300068704700F100607E
:100C1000920000F5803001F0EDBC0000054B1A6831
:100C2000054B1B789B1A834202D9104401F096BCF5
:100C300000207047802500209925002038B5074DF9
:100C400004462868204401F091FC28B92868204413
:100C5000BDE8384001F0A2BC38BD00BF80250020AF
:100C600010F0030308D1B0F5007F05D800F1005063
:100C7000A0F508400068704700207047014BC0583D
:100C8000704700BF107AFF1F014B1868704700BF04
:100C9000002004E070B52A4B1C68C4F30B03240C3D
:100CA00063B140F21342934231D040F21942934271
:100CB0002FD040F2214293422DD10323214A0C250B
:100CC00005FB03235D6893F9082042F201039C426F
:100CD00024D0B4F5805F23D041F201039C4221D09F
:100CE00041F203039C421FD041F207039C4208BF1C
:100CF0003122441E0C44013D0B46A3421ED215F97D
:100D0000016F581C96B1034600F8016CF5E701230A
:100D1000D4E70223D2E73F220B4DD6E73322E3E7A5
:100D20004122E1E75A22E4E75922E2E72C258442F6
:100D30001D7001D9981C5A70401A70BD1846FBE707
:100D4000002004E04C3B0008403B0008022802BFA2
:100D5000024B4FF080629A61704700BF000802406A
:100D6000022802BF024B4FF480629A61704700BFB5
:100D700000080240022801BF024A536983F48063DD
:100D8000536170470008024010B50023934203D01E
:100D9000CC5CC4540133F9E710BD000030B5441EEB
:100DA00014F9010F0B4660B193F90050854201F12F
:100DB000010106D11AB993F90020801A30BD013A19
:100DC000EEE7002AF7D1104630BD00000246034688
:100DD000981A13F9011B0029FAD1704702440346FF
:100DE000934202D003F8011BFAE77047024B1A78CE
:100DF000024B1A70704700BF982500200024002085
:100E0000F8B5184C1848194D194E174F00F0AAFCA8
:100E10002146154800F0D2FC24681648626DD2F8CD
:100E2000043843F00203C2F8043801F053F92046B5
:100E3000114900F0CFFD626DD2F8043823F00203AF
:100E4000C2F804384FF4E1332B60002456F8240034
:100E5000B84202D0294600F0E3FB0134042CF5D15E
:100E6000F8BD00BF643C0008A833002084250020A2
:100E70007C3B000840420F008C3C000838B50B4B0F
:100E80001A780B4B53F822400A4B9C4205460CD073
:100E9000094B002118461422FFF7A0FF0560014608
:100EA0002046BDE8384000F0BBBB38BD9825002087
:100EB0007C3B0008A83300208425002010B5054C99
:100EC000142200212046FFF789FF01236370024BA3
:100ED000636010BD9C2500200A080240FEE7000068
:100EE00000B59BB0EFF3098168226846FFF74CFF1D
:100EF000EFF30583034B9A6B9A6A9A6A9A6A9A6A25
:100F00009B6AFEE700ED00E000B59BB0EFF30981BE
:100F100068226846FFF738FFEFF30583044B9A6BAE
:100F20009A6A9A6A9A6A9A6A9A6A9B6AFEE700BF04
:100F300000ED00E000B59BB0EFF309816822684640
:100F4000FFF722FFEFF30583034B5A6B9A6A9A6A05
:100F50009A6A9A6A9B6AFEE700ED00E030B5084D98
:100F60000A4491420BD011F8013B09245840013C3E
:100F7000F7D040F300032B4083EA5000F7E730BD81
:100F80002083B8ED002304491A465A50C818083384
:100F9000802B4260F9D17047B02500200268436879
:100FA0001143016003B1184770470000024AD3683B
:100FB00043F0C003D360704700100140024AD36879
:100FC00043F0C003D360704700440040024AD36836
:100FD00043F0C003D3607047005000402DE9F0415A
:100FE000D0F85C64F7683368DA0505469CB20DD525
:100FF000202383F311884FF400710430FFF7CEFFF4
:101000006FF480733360002383F31188202383F30C
:10101000118805F1040814F02F0333D183F31188EC
:10102000380615D5210613D5202383F3118805F141
:10103000380000F053FA002846DA0821281DFFF78F
:10104000ADFF4FF67F733B40F360002383F31188BD
:101050007A060ED563060CD5202383F31188EA6C3B
:101060002B6D9A4202D12B6C002B2FD1002383F3DE
:101070001188D5F86424D368002B31D01069BDE8FD
:10108000F0411847230713D014F0080F0CBF0021BC
:101090008021E00748BF41F02001A20748BF41F08E
:1010A0004001630748BF41F480714046FFF776FF77
:1010B000A406736805D595F860142846194000F019
:1010C000BDFA3468A4B2A6E77060BEE727F0400717
:1010D0003F041021281D3F0CFFF760FFF760C5E7B4
:1010E000BDE8F08108B50348FFF778FFBDE8084088
:1010F00001F074BB3026002008B50348FFF76EFFEF
:10110000BDE8084001F06ABB982A002008B50348F2
:10111000FFF764FFBDE8084001F060BB002F00202E
:1011200010B50E4C0E4A2046002100F057FA0D4B28
:10113000C4F85C340C4C0D4A2046002100F04EFAF5
:101140000B4BC4F85C340B4C0B4A0021204600F0DA
:1011500045FA0A4BC4F85C3410BD00BF30260020AD
:10116000AD0F000800100140982A0020BD0F0008B4
:1011700000440040002F0020CD0F00080050004028
:1011800038B5394D037C002918BF0D46012B0446A4
:10119000C0F8645410D1354B984242D1344B5A6C4C
:1011A00042F010025A645A6E42F010025A665B6EA8
:1011B0000B21252000F06AF82E4BD4F85C249A42CB
:1011C0002B6802D02C498A424BD12C4901EB5301A8
:1011D000B1FBF3F3A988080442BF23F0070003F032
:1011E000070343EA40039360EB8843F040039BB25C
:1011F00013612B8943F001039BB2536141F4045303
:1012000043F02C03D36001F4A05100231360B1F527
:10121000806F136853680CBF7F23FF2384F860340A
:1012200038BD174B98420CD1114B1A6C42F4003266
:101230001A641A6E42F400321A661B6E0B212620C5
:10124000B8E7104B9842B7D1094B1A6C42F48012A0
:101250001A641A6E42F480121A661B6E0B21352036
:10126000A8E70949B2E700BFAC3B000830260020E0
:1012700000380240001001400014014000BD01058B
:10128000982A0020002F002080DE800200F16043B9
:1012900000F01F02400903F5614309018000C9B253
:1012A00000F1604083F8001300F561400123934092
:1012B000C0F8803103607047F8B51546826806694A
:1012C000AA420B46816938BF8568761AB542044642
:1012D00007D218462A46FFF757FDA3692B44A3619E
:1012E0000DE011D932461846FFF74EFDAF1B3A46C6
:1012F000E1683044FFF748FDE2683A44A261A36820
:101300005B1BA3602846F8BD18462A46FFF73CFD44
:10131000E368E4E783682DE9F0410446934215460B
:10132000266938BF85684069361AB5420F4606D22D
:101330002A46FFF729FD63692B4463610DE012D94A
:101340003246A5EB0608FFF71FFD4246B919E068D3
:10135000FFF71AFDE26842446261A3685B1BA36069
:101360002846BDE8F0812A46FFF70EFDE368E4E772
:1013700010B50A440024C361029B00604060846091
:10138000C160816141610261036210BD08B582697B
:101390004369934201D1826882B9826801328260D6
:1013A0005A1C42611970426903699A4201D3C368A9
:1013B0004361002100F0AAFE002008BD4FF0FF307D
:1013C00008BD000070B5202304460E4683F3118843
:1013D000A568A5B1A368A269013BA360531CA361E2
:1013E00015782269934224BFE368A361E3690BB1D6
:1013F00020469847002383F31188284670BD314664
:10140000204600F073FE0028E2DA85F3118870BDF3
:101410002DE9F74F05460F4690469A46D0F81C90A6
:10142000202686F311884FF0000B144664B1224643
:1014300039462846FFF740FF034668B9514628461B
:1014400000F054FE0028F1D0002383F31188A8EBAC
:10145000040003B0BDE8F08FB9F1000F03D0019094
:101460002846C847019B8BF31188E41A1F4486F372
:101470001188DBE7C16081614161C3611144009B58
:10148000006040608260016103627047F8B5044605
:101490000E461746202383F31188A568A5B1A368DB
:1014A000013BA36063695A1C62611E702369626913
:1014B0009A4224BFE3686361E3690BB12046984711
:1014C000002080F31188F8BD3946204600F00EFE5A
:1014D0000028E2DA85F31188F8BD000083694269CB
:1014E0009A4210B501D182687AB98268013282606D
:1014F0005A1C82611C7803699A4201D3C3688361D4
:10150000002100F003FE204610BD4FF0FF3010BD5B
:101510002DE9F74F05460F4690469A46D0F81C90A5
:10152000202686F311884FF0000B144664B1224642
:1015300039462846FFF7EEFE034668B9514628466D
:1015400000F0D4FD0028F1D0002383F31188A8EB2C
:10155000040003B0BDE8F08FB9F1000F03D0019093
:101560002846C847019B8BF31188E41A1F4486F371
:101570001188DBE7026843681143016003B1184733
:10158000704700001430FFF743BF00004FF0FF33F7
:101590001430FFF73DBF00003830FFF7B9BF00003F
:1015A0004FF0FF333830FFF7B3BF00001430FFF7C0
:1015B00009BF00004FF0FF311430FFF703BF0000F8
:1015C0003830FFF763BF00004FF0FF323830FFF7CD
:1015D0005DBF000000207047FFF7A2BD37B50F4B7D
:1015E0000360002343608360C360012304460374E7
:1015F000154600900B464FF4007200F15C01143068
:10160000FFF7B6FE00942B464FF4007204F51771F5
:1016100004F13800FFF72EFF03B030BDC03B0008D7
:1016200010B52023044683F31188FFF7A9FD022398
:101630002374002383F3118810BD000038B5C369FB
:1016400004460D461BB904210844FFF793FF2946C1
:1016500004F11400FFF79AFE002806DA201D4FF46B
:101660008061BDE83840FFF785BF38BD0268436838
:101670001143016003B118477047000013B5446B74
:10168000D4F894341A681178042915D1217C0229E0
:1016900012D11979128901238B4013420CD101A96F
:1016A00004F14C0001F050FED4F89444019B2179E0
:1016B0000246206800F0DAF902B010BD143001F0E3
:1016C000D3BD00004FF0FF33143001F0CDBD00005A
:1016D0004C3001F0A5BE00004FF0FF334C3001F05C
:1016E0009FBE0000143001F0A1BD00004FF0FF319B
:1016F000143001F09BBD00004C3001F071BE0000C1
:101700004FF0FF324C3001F06BBE0000D0F8942453
:1017100038B5136819780429054601D0012038BD71
:10172000017C0229FAD112795C89012090400440A1
:10173000F4D105F1140001F033FD02460028EDD08C
:10174000D5F894544FF480732868697900F07CF9D7
:10175000204638BD406BFFF7D9BF0000002070471E
:10176000704700007FB5124B036000234360836025
:10177000C360012502260F4B0574044602900193B5
:1017800000F18402294600964FF48073143001F072
:10179000E3FC094B0193029400964FF4807304F527
:1017A0002372294604F14C0001F0AAFD04B070BD7B
:1017B000E83B0008551700087D1600080B6820223A
:1017C00082F311880A7903EB820290614A79093227
:1017D00043F822008A7912B103EB82039861022355
:1017E0000374C0F89414002383F311887047000039
:1017F00038B5037F044613B190F85430ABB9201DBF
:1018000001250221FFF732FF04F1140025776FF064
:10181000010100F087FC84F8545004F14C006FF093
:101820000101BDE8384000F07DBC38BD10B5012194
:1018300004460430FFF71AFF0023237784F854305E
:1018400010BD000038B504460025143001F09CFCA2
:1018500004F14C00257701F06BFD201D84F85450F5
:101860000121FFF703FF2046BDE83840FFF74EBFD8
:1018700090F8443003F06003202B19D190F84520F4
:10188000212A0AD0222A4FF000030ED0202A0FD19D
:10189000084A82630722C26304E0064B836307237E
:1018A000C36300230364012070478363C363F9E7C4
:1018B0000020704701240020D0F8943437B51A680E
:1018C0001178042904461AD1017C022917D119790B
:1018D000128901238B40134211D100F14C05284697
:1018E00001F0E6FD58B101A9284601F02DFDD4F81C
:1018F0009444019B21790246206800F0B7F803B0B8
:1019000030BD000000EB8103F7B59C6905460E462B
:10191000F4B1202383F3118805EB8607201D0821ED
:10192000FFF7A4FEFB685B691B684C3413B12046CB
:1019300001F018FD01A9204601F006FD024648B15C
:10194000019B3146284600F091F8002383F311886B
:1019500003B0F0BDFB685A691268002AF5D01B8AF3
:10196000013B1340F1D105F14402EAE7093138B5F2
:1019700050F82140DCB1202383F31188D4F894245B
:101980001368527903EB8203DB689B695D6845B19C
:1019900004216018FFF76AFE294604F1140001F0E3
:1019A00009FC2046FFF7B2FE002383F3118838BDFF
:1019B0007047000000F0CABF01230370002343609A
:1019C000C36183620362C362436203630381438131
:1019D0007047000038B50446202383F311880025A2
:1019E0004160C56005614561856100F0BFFF02236C
:1019F000237085F3118838BD70B500EB810305466F
:101A00005069DA600E46144618B110220021FFF723
:101A1000E5F9A06918B110220021FFF7DFF931467E
:101A20002846BDE8704001F06BB80000028902F062
:101A300001020281428902F0010242810022026118
:101A40004261826101F0F0B8F0B400EB8104478993
:101A5000E4680125A4698D403D434581236000234E
:101A6000A2606360F0BC01F00BB90000F0B400EBC1
:101A700081040789E468012564698D403D4305813F
:101A800023600023A2606360F0BC01F085B9000010
:101A900070B50223002504460370A0F84C5080F86E
:101AA0004E5080F84F5005814581C5600561456104
:101AB000856180F8345000F0BFFF63681B6823B174
:101AC00029462046BDE87040184770BD436802783B
:101AD0001B6880F85020052202700BB104211847C2
:101AE00070470000436890F850201B6802700BB1EB
:101AF000052118477047000090F8343070B504464F
:101B000013B1002380F8343004F14402204601F080
:101B1000ADF863689B6863BB94F8445015F06006A9
:101B200015D194F8453005F07F0545EA032540F2CC
:101B300002339D4200F00E815BD8022D00F0DC8064
:101B40003FD8002D00F08780012D00F0CF800021CC
:101B5000204601F0E3FA0021204601F0D5FA63683F
:101B60001B6813B1062120469847062384F83430B9
:101B700070BD204698470028CED094F84B2094F8AA
:101B80004A3043EA0223E26B934238BFE36394F99D
:101B90004430E56B002B4FF0200380F2FD80002DD8
:101BA00000F0EC80092284F8342083F311880021AE
:101BB000E36BA26B2046FFF759FF002383F31188E4
:101BC00070BDB5F5817F00F0B180B5F5407F49D09B
:101BD000B5F5807FBBD194F84630012BB7D1B4F86E
:101BE0004C3023F00203A4F84C30A663E66326646D
:101BF000C3E740F201639D421ED8B5F5C06F3BD2EA
:101C0000B5F5A06FA3D1B4F84430B3F5A06F0ED1F1
:101C100094F8463084F84E30204600F065FF636843
:101C20001B6813B10121204698470323237000232A
:101C3000A363E3632364A0E7B5F5106F32D040F6E9
:101C400002439D4252D0B5F5006F80D104F14F039D
:101C5000A363012324E004F14C03A3630223E363A1
:101C600025648AE794F84630012B7FF470AFB4F80E
:101C70004C3043F00203B6E794F84920616894F8C9
:101C800048304D6894F8471043EA0223204694F800
:101C90004620A84700283FF45AAF4368A36303686F
:101CA000E363A4E72378042B10D1202383F3118866
:101CB0002046FFF7BBFE86F31188636884F84F6007
:101CC0001B68032121700BB12046984794F84630D9
:101CD000002BACD084F84F300423237063681B685A
:101CE000002BA4D0022120469847A0E7374BA363DE
:101CF0000223E36300239DE794F8481011F0800F5E
:101D0000204601F00F010ED000F0A2FF012806D0FE
:101D100002287FF41CAF2E4BA363E06367E72D4BD3
:101D2000A363E56363E700F085FFEFE794F84630CF
:101D3000002B7FF40CAF94F8483013F00F013FF400
:101D400076AF1A06204602D501F0FCF96FE701F0E4
:101D5000EFF96CE794F84630002B7FF4F8AE94F876
:101D6000483013F00F013FF462AF1B06204602D546
:101D700001F0D4F95BE701F0C7F958E7142284F8C1
:101D8000342083F311882B462A4629462046FFF744
:101D90005BFE85F3118870BD5DB1152284F8342097
:101DA00083F311880021E36BA26B2046FFF74CFE02
:101DB00003E70B2284F8342083F311882B462A464C
:101DC00029462046FFF752FEE3E700BF183C000813
:101DD000103C0008143C000838B590F83430044634
:101DE000152B29D8DFE803F03E28282828283E288C
:101DF000280B293928282828282828283E3E90F80A
:101E00004B1090F84A20C36B42EA01229A4214D93F
:101E1000C268128AB3FBF2F502FB15356DB92023B7
:101E200083F311882B462A462946FFF71FFE85F3C8
:101E300011880A2384F8343038BD142384F83430F0
:101E4000202383F3118800231A4619462046FFF702
:101E5000FBFD002383F3118838BD036C03B1984761
:101E60000023E7E7002101F059F90021204601F0A5
:101E70004BF963681B6813B1062120469847062377
:101E8000D8E7000090F83420152A38B5044622D847
:101E90000123934040F6416213421DD113F4801593
:101EA0000FD19B0217D50B2380F83430202383F306
:101EB00011882B462A462946FFF7D8FD85F311885D
:101EC00038BDC3689B695B682BB9036C03B1984745
:101ED000002384F8343038BD002101F01FF90021BF
:101EE000204601F011F963681B6813B106212046F2
:101EF00098470623EDE70000024B00221B605B6061
:101F00009A60704768330020002303748268054B91
:101F10001B6899689142FBD25A6803604260106066
:101F2000586070476833002008B5202383F3118878
:101F3000037C032B05D0042B0DD02BB983F3118820
:101F400008BD436900221A604FF0FF334361FFF779
:101F5000DBFF0023F2E790E80C001A600268536090
:101F6000F2E70000002303748268054B1B68996840
:101F70009142FBD85A680360426010605860704715
:101F800068330020054B19690874186802681A60E4
:101F90005360186101230374FEF7B8B96833002059
:101FA00030B54B1C87B005460A4C10D023690A4A4D
:101FB00001A800F0D3F82846FFF7E4FF049B13B113
:101FC00001A800F007F92369586907B030BDFFF791
:101FD000D9FFF8E768330020291F000838B50C4DF9
:101FE00041612B6981689A689142044603D8BDE833
:101FF0003840FFF789BF1846FFF786FF01232C61A1
:10200000014623742046BDE83840FEF77FB900BF83
:1020100068330020044B1A681B6990689B689842DB
:1020200094BF0020012070476833002010B5084C91
:10203000236820691A6822605460012223611A749F
:10204000FFF790FF01462069BDE81040FEF75EB93A
:1020500068330020826002220274002242747047BA
:102060008368A3F17C0243F80C2C026943F83C2CF2
:10207000426943F8382C074A43F81C2CC26843F8DD
:10208000102C022203F8082C002203F8072CA3F1DD
:10209000180070472503000810B5202383F311882A
:1020A000FFF7DEFF00210446FFF798FF002383F3CC
:1020B0001188204610BD0000024B1B6958610F209B
:1020C000FFF760BF68330020202383F31188FFF7F8
:1020D000F3BF000008B50146202383F311880820D0
:1020E000FFF75EFF002383F3118808BD49B1064B5B
:1020F00042681B6918605A60136043600420FFF750
:102100004FBF4FF0FF30704768330020036898429C
:1021100006D01A680260506059611846FFF7F4BE95
:102120007047000038B504460D462068844200D14F
:1021300038BD036823605C604561FFF7E5FEF4E7A6
:10214000054B03F114025A619A614FF0FF32DA61D4
:1021500000221A62704700BF68330020F8B503619F
:102160004FF08043C2605C6A194B1A46022952F84C
:10217000145F38BF0221954206461F460AD15861B6
:1021800098611C620560456081600819BDE8F840EF
:1021900001F0B0B9186AAB68241A0C1902D3E41A1A
:1021A0002D6804E09C4202D2204401F0B1F9AB68F2
:1021B0009C42F4D86B68736035601E606E60B460DA
:1021C000A9684FF0FF33091BA960FB61F8BD00BF90
:1021D0006833002010B41B4C234653F8141F81426F
:1021E00010D0416802680A60026851609A424FF05C
:1021F0000001C16003D0936881680B4493605DF86F
:10220000044B70470A68626100209A425360C860BC
:1022100003D15DF8044B01F075B9936888680344F5
:1022200093604FF08042206A526A121A9342E6D9B4
:10223000991A012998BF931C18445DF8044B01F0CA
:1022400067B900BF6833002000207047FEE7000038
:10225000704700004FF0FF3070470000022906D0A1
:10226000032906D00129064818BF002070470548F9
:102270007047032A9ABF044800EBC2000020704751
:10228000E83C00089C3C00080824002070B59AB087
:1022900001AD064608462946144600F095F8284642
:1022A000FEF794FDC0B2431C5B0086E81800237063
:1022B00003236370002302341946DAB2904204F11A
:1022C000020401D81AB070BDEA5C04F8022C04F8CC
:1022D000011C0133F1E7000008B5202383F31188C6
:1022E0000348FFF7E9FA002383F3118808BD00BF14
:1022F000A833002010B50446052916D8DFE801F000
:1023000016150316161D202383F311880E4A01218A
:10231000FFF772FB20460D4A0221FFF76DFB0C48C8
:10232000FFF790FA002383F3118810BD202383F375
:1023300011880748FFF75CFAF4E7202383F311883C
:102340000348FFF773FAEDE71C3C0008403C000827
:10235000A833002038B50C4D0C4C0D492A4604F129
:102360000800FFF793FF05F1CA0204F110000949C4
:10237000FFF78CFF05F5CA7204F118000649BDE8A5
:102380003840FFF783BF00BF7038002008240020CA
:102390006C3C0008763C0008813C000870B504469F
:1023A00008460D46FEF712FDC6B2204601340378FA
:1023B0000BB9184670BD32462946FEF7EFFC0028DF
:1023C000F3D1012070BD00002DE9F84F05460C4601
:1023D000FEF7FCFC2B49C6B22846FFF7DFFF08B129
:1023E0000536F6B228492846FFF7D8FF08B110365F
:1023F000F6B2632E0DD8DFF88C80DFF88C90234F77
:10240000DFF890A0DFF890B02E7846B92670BDE8CE
:10241000F88F29462046BDE8F84F01F085BB252EF0
:102420002CD1072241462846FEF7B8FC58B9DBF804
:1024300000302360DBF804306360DBF80830A36011
:1024400007350C34E0E7082249462846FEF7A6FC8B
:10245000A0B90F4BA21C13F8011F09095345C95D10
:1024600002F8021C197801F00F0102F10202C95DA5
:1024700002F8031CEFD118340835C5E72670013582
:102480000134C1E7083D0008813C00081D3D0008FB
:102490000F7AFF1F1B7AFF1F103D0008BFF34F8FFD
:1024A000024AD368DB03FCD4704700BF003C024003
:1024B00008B5094B1B7873B9FFF7F0FF074B1A6992
:1024C000002ABFBF064A5A6002F188325A601A6871
:1024D00022F480621A6008BDCE3A0020003C02401F
:1024E0002301674508B50B4B1B7893B9FFF7D6FF5F
:1024F000094B1A6942F000421A611A6842F480528C
:102500001A601A6822F480521A601A6842F48062D3
:102510001A6008BDCE3A0020003C02400B2870B57E
:1025200013D80B4A0B4C137863B90B4E4FF0006174
:1025300044F8231056F8235001330C2B2944F7D1CB
:102540000123137054F8200070BD002070BD00BF3F
:10255000003B0020D03A0020303D0008014B53F8EA
:1025600020007047303D00080C2070470B2810B544
:10257000044601D9002010BDFFF7D0FF064B53F8E9
:1025800024301844C21A0BB9012010BD1268013260
:10259000F0D1043BF6E700BF303D00080B2810B532
:1025A000044621D8FFF77AFFFFF782FF0F4AF32393
:1025B000D360C300DBB243F4007343F00203136142
:1025C000136943F480331361FFF768FFFFF7A6FF39
:1025D000074B53F8241000F0DDF8FFF783FF204687
:1025E000BDE81040FFF7C2BF002010BD003C024014
:1025F000303D00082DE9F84312F00103154640D1A3
:102600008218B2F1016F3CD22C4B1B6813F001030E
:1026100037D02B4CFFF74CFFF323E360FFF73EFF6F
:1026200040F20127032D01D9830713D0244C0F4614
:10263000401A40F20118EB1B0B44012B00EB07067C
:10264000236924D823F001032361FFF74BFF012006
:10265000BDE8F883236923F44073236123693B4376
:10266000236151F8046B0660BFF34F8FFFF716FF2D
:1026700003689E4208D0236923F001032361FFF71A
:1026800031FF0020BDE8F883043D0430CAE723F49D
:1026900040732361236943EA08032361B94637F88D
:1026A000023B3380BFF34F8FFFF7F8FE3688B9F84F
:1026B0000030B6B2B342BED0DDE700BF0038024002
:1026C000003C0240084908B50B7828B153B9FFF720
:1026D000EFFE01230B7008BD23B1BDE80840087070
:1026E000FFF700BF08BD00BFCE3A002010B502447E
:1026F000064B0439D2B2904200D110BD441C00B246
:1027000053F8200041F8040FE0B2F4E750280040ED
:10271000104B30B51C6F240407D41C6F44F40074B4
:102720001C671C6F44F400441C670B4C236843F483
:10273000807323600244094B0439D2B2904200D125
:1027400030BD441C00B251F8045F43F82050E0B2A1
:10275000F4E700BF003802400070004050280040FD
:1027600007B5012201A90020FFF7C0FF019803B0BF
:102770005DF804FB13B50446FFF7F2FFA04206D054
:1027800002A9012241F8044D0020FFF7C1FF02B069
:1027900010BD000070470000034B1B689B0042BF48
:1027A000024B01221A70704774380240013B00202E
:1027B000014B1878704700BF013B0020064A536860
:1027C00023F001035360EFF30983683383F309882F
:1027D000002383F31188704730EF00E010B5202309
:1027E00083F31188104B5B6813F4006318D0F1EE8B
:1027F000103AEFF309844FF0807344F84C3C0B4BD4
:10280000DB6844F8083CA4F1680383F30988FFF708
:1028100001FC18B1064B44F8503C10BD054BFAE7DB
:1028200083F3118810BD00BF00ED00E030EF00E041
:10283000350300083803000870470000FEE7000079
:10284000084A094B09498B4204D3094A00219342A3
:1028500005D3704752F8040F43F8040BF3E743F82D
:10286000041BF4E7DC3E0008783D0020783D0020A2
:10287000783D0020836D30B500229D68446D11467F
:102880004FF0FF3004EB421301329542C3F80019B8
:10289000C3F81019C3F80809C3F8001BC3F8101BCC
:1028A000C3F8080BEED24FF00113C4F81C3830BD4A
:1028B000890141F02001016103699B06FCD41220CB
:1028C00000F0AEBE204B03EB80022DE9F047D2F8BA
:1028D0000CE05D6DDEF81420461CD2F800C005EB5C
:1028E000063605EB4018516861450BD3D5F83428FE
:1028F000012303FA00F022EA0000C5F83408184664
:10290000BDE8F087BEF81040ACEB0103A34228BF3E
:102910002346D8F81849A4B2B3EB840F10D89468B2
:102920001F46A4F1040959F804AFC6F800A0042F0B
:1029300001D9043FF7E71C440B4494605360D2E78D
:102940000020BDE8F08700BF043B002010B5054C17
:102950002046FFF731F84FF0A0436365024BA365B3
:1029600010BD00BF043B0020843D00080378012B0C
:1029700070B5054650D12A4B446D98421BD1294B66
:102980005A6B42F080025A635A6D42F080025A65D7
:102990005A6D5A6942F080025A615A6922F08002E7
:1029A0005A610E2143205B69FEF770FC1E4BE36009
:1029B0001E4BC4F800380023C4F8003EC023236037
:1029C0006E6D4FF40413A3633369002BFCDA01230B
:1029D00033610C2000F024FE3369DB07FCD41220A5
:1029E00000F01EFE3369002BFCDA0026A6602846A4
:1029F000FFF740FF6B68C4F81068DB68C4F8146820
:102A0000C4F81C684BB90A4BA3614FF0FF336361F4
:102A1000A36843F00103A36070BD064BF4E700BF59
:102A2000043B002000380240401400400300200214
:102A3000003C30C0083C30C0F8B5446D054600216C
:102A40002046FFF735FFA96D00234FF001128F6874
:102A5000C4F834384FF00066C4F81C284FF0FF303B
:102A600004EB431201339F42C2F80069C2F8006BC5
:102A7000C2F80809C2F8080BF2D20B686A6DEB6560
:102A8000636210231361166916F01006FBD1122041
:102A900000F0C6FDD4F8003823F4FE63C4F8003813
:102AA000A36943F4402343F01003A3610923C4F84E
:102AB0001038C4F814380A4BEB604FF0C043C4F828
:102AC000103B084BC4F8003BC4F81069C4F8003947
:102AD000EB6D03F1100243F48013EA65A362F8BDC5
:102AE000603D000840800010426D90F84E10D2F812
:102AF000003823F4FE6343EA0113C2F8003870473C
:102B00002DE9F0410EB200EB86080D46D8F80C1006
:102B10000F6807F00303022B50D0032B50D03D4A1F
:102B20003D4F012B18BF1746446D4FEA451E04EB7D
:102B30000E030022C3F8102B8A6905F1100C002A3D
:102B400040D04A8A05F158035B013A43E250012321
:102B5000D4F81C2803FA0CF31343A6444A69C4F8BA
:102B60001C380023CEF8103905F13F03002A39D074
:102B70000A8A898B9208012988BF4A43C16D04EBF8
:102B80008303561841EA0242C66529465A60204628
:102B9000FFF78EFED8F80C301B8A43EA85531F439B
:102BA00005F148035B01E7500123D4F81C2803FA20
:102BB00005F51543C4F81C58BDE8F081174FB3E77D
:102BC000174FB1E704EB4613D3F8002B22F4004271
:102BD000C3F8002BD4F81C28012303FA0CF322EAD3
:102BE0000303BAE704EB83030E4A5A6004EB46166C
:102BF00029462046FFF75CFED6F8003923F400434F
:102C0000C6F80039D4F81C38012202FA05F523EA87
:102C10000505CFE700800010008004100080081038
:102C200000800C1000040002826D1268C265FFF77C
:102C300021BE00005831436D49015B5813F4004038
:102C400004D013F4001F14BF0120022070470000BD
:102C50004831436D49015B5813F4004004D013F42C
:102C6000001F14BF012002207047000000EB81010B
:102C7000CB68196A0B6813604B685360704700009B
:102C800000EB810330B5DD68AA691368D36019B918
:102C9000402B84BF402313606B8A1468426D1C4430
:102CA000013CB4FBF3F46343033323F0030302EB6F
:102CB000411043EAC44343F0C043C0F8103B2B68C3
:102CC00003F00303012B09B20ED1D2F8083802EB4E
:102CD000411013F4807FD0F8003B14BF43F08053C1
:102CE00043F00053C0F8003B02EB4112D2F8003B26
:102CF00043F00443C2F8003B30BD00002DE9F04131
:102D0000244D6E6D06EB40130446D3F8087BC3F8E0
:102D1000087B38070AD5D6F81438190706D505EB0D
:102D200084032146DB6828465B689847FA072FD55D
:102D3000D6F81438DB072BD505EB8403D968CCB95A
:102D40008B69488A5E68B6FBF0F200FB12628AB9B2
:102D50001868DA6890420DD2121A83E81400202312
:102D600083F311880B482146FFF78AFF84F311880B
:102D7000BDE8F081012303FA04F26B8923EA020320
:102D80006B81CB6823B121460248BDE8F04118476A
:102D9000BDE8F081043B002000EB810370B5DD68E5
:102DA000436D6C692668E6604A0156BB1A444FF4CD
:102DB0000020C2F810092A6802F00302012A0AB2B0
:102DC0000ED1D3F8080803EB421410F4807FD4F836
:102DD000000914BF40F0805040F00050C4F80009D2
:102DE00003EB4212D2F8000940F00440C2F8000997
:102DF000D3F83408012202FA01F10143C3F8341870
:102E000070BD19B9402E84BF4020206020682E8AF2
:102E1000841940F00050013C1A44B4FBF6F440EA37
:102E2000C440C6E7F8B504461E48456D05EB44139B
:102E3000D3F80869C3F80869F10717D5D5F8103831
:102E4000DA0713D500EB8403D9684B691F68DA6889
:102E5000974218D2D21B00271A605F60202383F3A9
:102E600011882146FFF798FF87F31188330617D59D
:102E7000D5F834280123A340134211D02046BDE8E1
:102E8000F840FFF71FBD012303FA04F2038923EA88
:102E9000020303818B68002BE8D021469847E5E7C1
:102EA000F8BD00BF043B002096482DE9F84F456D62
:102EB0006E69AB691E4016F4805F6E61044605D0F2
:102EC000FEF7E6FDBDE8F84FFFF788BC002E12DAEA
:102ED000D5F8003E8B489B071EBFD5F8003E23F077
:102EE0000303C5F8003ED5F8043823F00103C5F804
:102EF0000438FEF7F7FD370502D58248FEF7E6FDF8
:102F0000B0040CD5D5F8083813F0060FEB6823F49D
:102F100070530CBF43F4105343F4A053EB603107DC
:102F200004D56368DB680BB176489847F2025AD43F
:102F3000B3020CD5D4F85480DFF8C8A100274FF0B5
:102F40000109A36D9B68F9B28B4280F08780F70678
:102F500019D5616D0A6AC2F30A1702F00F0302F471
:102F6000F012B2F5802F00F0A180B2F5402F0AD107
:102F700004EB830301F58051DB68186A00231A46CD
:102F80009F4240F087803003D5F8184813D5E103FD
:102F900002D50020FFF7B2FEA20302D50120FFF701
:102FA000ADFE630302D50220FFF7A8FE270302D57A
:102FB0000320FFF7A3FE750384D5E00702D50020A8
:102FC000FFF730FFA10702D50120FFF72BFF6207B3
:102FD00002D50220FFF726FF23077FF573AF0320FA
:102FE000FFF720FF6EE7D4F85480DFF818A1002720
:102FF0004FF00109A36D9B685FFA87FB5B4597D390
:1030000008EB4B13D3F8002902F44022B2F5802FCD
:1030100022D1D3F80029002A1EDAD3F8002942F081
:103020009042C3F80029D3F80029002AFBDB594657
:10303000606DFFF73DFC228909FA0BF322EA0303D6
:10304000238104EB8B03DB689B6813B15946504620
:1030500098475846FFF736FC0137CBE708EB41129B
:10306000D2F8003B03F44023B3F5802F10D1D2F8FF
:10307000003B002B0CDA628909FA01F322EA030310
:10308000638104EB8103DB68DB680BB15046984732
:10309000013756E79C0708BF0A68072B98BF0270E4
:1030A00003F101039CBF120A013069E7023304EB0C
:1030B000830201F58051526890690268D0F808C017
:1030C0004068A2EB000E0022104697420AD104EBA2
:1030D000830463689B699A683A449A605A68174403
:1030E0005F6050E712F0030F08BF0868964588BF7D
:1030F0008CF8000002F1010284BF000A0CF1010CFF
:10310000E3E700BF043B0020436D03EB4111D1F81E
:10311000003B43F40013C1F8003B7047436D03EBE1
:103120004111D1F8003943F40013C1F80039704758
:10313000436D03EB4111D1F8003B23F40013C1F8B8
:10314000003B7047436D03EB4111D1F8003923F484
:103150000013C1F80039704730B5039C0172043385
:1031600004FB0325C361049B03630021059B0060EE
:103170004060C160426102618561046242628162B5
:10318000C162436330BD00000022416A41610161B8
:10319000C2608262C2626FF00101FEF7C3BF00002D
:1031A00003694269934203D1C2680AB100207047A3
:1031B000181D704703691960C2680132C260C26994
:1031C000134482690361934224BF436A036100216F
:1031D000FEF79CBF38B504460D46E3683BB1626913
:1031E000131D1268A3621344E362002038BD237AE2
:1031F00033B929462046FEF779FF0028EDDA38BDBD
:103200006FF00100FBE70000C368C269013BC360C7
:103210004369134482694361934224BF436A436113
:1032200000238362036B03B11847704770B52023F6
:10323000044683F31188866A3EB9FFF7CBFF054643
:1032400018B186F31188284670BDA36AE26A13F8A4
:10325000015BA362934202D32046FFF7D5FF002310
:1032600083F31188EFE700002DE9F84F04460E467E
:1032700090469946202787F311880025AA46D4F85E
:1032800028B0BBF1000F09D149462046FFF7A2FF45
:1032900020B18BF311882846BDE8F88FA16AE36A54
:1032A000A8EB050B5B1A9B4528BF9B46BBF1400F63
:1032B0001BD9334601F1400251F8040B43F8040BCB
:1032C0009142F9D1A36A40334036A3624035A26AE5
:1032D000E36A9A4202D32046FFF796FF8AF31188E9
:1032E0004545D8D287F31188C9E730465A46FDF7DD
:1032F0004BFDA36A5B445E44A3625D44E7E70000C4
:1033000010B5029C0172043303FB0421C361002346
:103310008362C362039B0363049B00604060C460DC
:1033200042610261816104624262436310BD000038
:10333000026AC260426A4261026100228262C26223
:103340006FF00101FEF7EEBE436902699A4203D1B4
:10335000C2680AB100207047184650F8043B0B6061
:1033600070470000C368C2690133C36043691344F6
:1033700082694361934224BF436A43610021FEF79F
:10338000C5BE000038B504460D46E3683BB123696D
:103390001A1DA262E2691344E362002038BD237A59
:1033A00033B929462046FEF7A1FE0028EDDA38BDE4
:1033B0006FF00100FBE7000003691960C268013A81
:1033C000C260C269134482690361934224BF436AA5
:1033D000036100238362036B03B118477047000049
:1033E00070B5202304460E4683F31188856A35B9EB
:1033F0001146FFF7C7FF10B185F3118870BDA36AAE
:103400001E70A36AE26A01339342A36204D3E169A6
:1034100020460439FFF7D0FF002080F3118870BDEB
:103420002DE9F84F04460D4691469A464FF0200884
:1034300088F311880026B346A76A4FB95146204643
:10344000FFF7A0FF20B187F311883046BDE8F88F61
:10345000A06AE76AA9EB06033F1A9F4228BF1F46EE
:10346000402F1BD905F1400355F8042B40F8042BDD
:103470009D42F9D1A36A4033A3624036A26AE36A4F
:103480009A4204D3E16920460439FFF795FF8BF394
:1034900011884E45D9D288F31188CDE729463A469E
:1034A000FDF772FCA36A3B443D44A3623E44E5E75A
:1034B000026943699A4203D1C3681BB91846704731
:1034C0000023FBE7836A002BF8D0043B9B1AF5D05E
:1034D0001360C368013BC360C3691A448369026116
:1034E0009A4224BF436A0361002383620123E5E714
:1034F00000F02EB94FF08043002258631A61022277
:10350000DA6070474FF080430022DA6070470000B5
:103510004FF0804358637047FEE7000010B5174C2A
:10352000FEF7EAFCFEF70CFE802215492046FEF766
:1035300091FD012344F8180C0374124B124AD96808
:1035400021F4E0610904090C0A431049DA60CA68F1
:1035500042F08072CA600E490A6842F001020A60B5
:103560001022DA77202283F82220002383F31188A7
:1035700062B60848BDE81040FEF78EBD90330020CB
:10358000903D000800ED00E00003FA05F0ED00E0DA
:10359000001000E0983D00082DE9F84F1F4C4FF057
:1035A0000008656904F11407C1464FF08043266A9C
:1035B0005B6AAA689E1B96421DD34FF0200AAA6838
:1035C000236AD5F80CB0134423622B68BB425F60BA
:1035D000A6EB02066361C5F80C8001D1FFF792FFEC
:1035E00089F311882869D8478AF311886569AB681F
:1035F0009E42E4D2D9E76269BA420CD09168236254
:103600008E1B9660A86802282CBF1818981CBDE86D
:10361000F84FFFF77DBFBDE8F88F00BF683300208B
:10362000034B59685A68521A9042FBD8704700BF42
:10363000001000E04B6843608B688360CB68C36018
:103640000B6943614B6903628B6943620B680360DA
:103650007047000008B5224B22481A6940F2FF115A
:103660000A431A611A6922F4FF7222F001021A61F8
:103670001A691A6B0A431A631A6D0A431A651A4AC1
:103680001B6D1146FFF7D6FF184802F11C01FFF72A
:10369000D1FF174802F13801FFF7CCFF154802F1BE
:1036A0005401FFF7C7FF144802F17001FFF7C2FF92
:1036B000124802F18C01FFF7BDFF114802F1A80189
:1036C000FFF7B8FF0F4802F1C401FFF7B3FF0E4840
:1036D00002F1E001FFF7AEFFBDE8084000F0A2B83C
:1036E0000038024000000240B83D000800040240DB
:1036F00000080240000C024000100240001402408A
:1037000000180240001C02400020024008B500F0F2
:10371000F9F9FFF703FFFFF73FF8BDE80840FEF7B0
:1037200019BE0000704700004FF0804310B51A69C1
:10373000920708D500241C61202383F31188FFF72A
:103740002BFF84F31188BDE81040FFF747B8000055
:10375000104B1A6C42F001021A641A6E42F0010218
:103760001A660D4A1B6E936843F0010393604FF095
:10377000804353229A624FF0FF32DA6200229A614C
:103780005A63DA605A6001225A6108211A601C20CB
:10379000FDF77CBD00380240002004E01F4B1A6991
:1037A0006FEAC2526FEAD2521A611A69C2F3080272
:1037B0001A614FF0FF301A695A69586100215A693D
:1037C00059615A691A6A62F080521A621A6A02F0E2
:1037D00080521A621A6A5A6A58625A6A59625A6A56
:1037E0001A6C42F080521A641A6E42F080521A66C5
:1037F0001A6E0B4A106840F480701060186F00F465
:103800004070B0F5007F1EBF4FF480301867196715
:10381000536823F40073536000F054B90038024039
:1038200000700040304B4FF080521A642F4A4FF422
:10383000404111601A6842F001021A601A6892074A
:10384000FCD59A6822F003029A60274B19469A68C1
:1038500012F00C02FBD1186800F0F90018609A60B1
:103860001A6842F480321A600B689B03FCD54B6FD8
:1038700043F001034B671C4B5A6F9007FCD51C4A61
:103880005A601A6842F080721A60184A53685904E4
:10389000FCD5154B1A689201FCD5164A9A60164B56
:1038A0001A68164B9A42164B1BD1164A1168164AD3
:1038B000914216D140F205121A600B4B9A6842F001
:1038C00002029A609A6802F00C02082AFAD15A6C35
:1038D00042F480425A645A6E42F480425A665B6EE9
:1038E000704740F20572E7E7003802400070004080
:1038F0000854400700948838002004E01164002038
:10390000003C024000ED00E041C20F41084A08B50A
:10391000536911680B4003F00103536123B1054A59
:1039200013680BB150689847BDE80840FEF756BFD2
:10393000003C0140B0250020084A08B553691168D1
:103940000B4003F00203536123B1054A93680BB1A6
:10395000D0689847BDE80840FEF740BF003C0140F2
:10396000B0250020084A08B5536911680B4003F0E0
:103970000403536123B1054A13690BB15069984799
:10398000BDE80840FEF72ABF003C0140B0250020FA
:10399000084A08B5536911680B4003F008035361E6
:1039A00023B1054A93690BB1D0699847BDE8084037
:1039B000FEF714BF003C0140B0250020084A08B5BE
:1039C000536911680B4003F01003536123B1054A9A
:1039D000136A0BB1506A9847BDE80840FEF7FEBE77
:1039E000003C0140B0250020174B10B55C691A68F7
:1039F000144004F478725A61A30604D5134A936AFA
:103A00000BB1D06A9847600604D5104A136B0BB10E
:103A1000506B9847210604D50C4A936B0BB1D06BC1
:103A20009847E20504D5094A136C0BB1506C9847CE
:103A3000A30504D5054A936C0BB1D06C9847BDE83B
:103A40001040FEF7CBBE00BF003C0140B025002077
:103A50001A4B10B55C691A68144004F47C425A6130
:103A6000620504D5164A136D0BB1506D98472305B6
:103A700004D5134A936D0BB1D06D9847E00404D57B
:103A80000F4A136E0BB1506E9847A10404D50C4A2F
:103A9000936E0BB1D06E9847620404D5084A136F39
:103AA0000BB1506F9847230404D5054A936F0BB1AF
:103AB000D06F9847BDE81040FEF790BE003C014033
:103AC000B0250020062108B50846FDF7DFFB0621DA
:103AD0000720FDF7DBFB06210820FDF7D7FB0621B9
:103AE0000920FDF7D3FB06210A20FDF7CFFB0621B5
:103AF0001720FDF7CBFB06212820BDE80840FDF785
:103B0000C5BB000008B5FFF749FEFDF73BFAFDF71E
:103B100063FDFDF74FFFFDF723FEFFF703FEBDE852
:103B20000840FFF7E5BC0000034611F8012B03F83D
:103B3000012B002AF9D17047121012131211000044
:103B400053544D3332463F3F3F0000000000000019
:103B5000403B00083F000000130400008C3B0008BD
:103B60003F00000019040000963B00083F000000E1
:103B700021040000A03B00083F000000A833002003
:103B800030260020982A0020002F002053544D3367
:103B900032463430780053544D3332463432780054
:103BA00053544D3332463434365858000096000092
:103BB0000000000000000000000000000000000005
:103BC00000000000A11500088D150008C9150008A7
:103BD000B5150008C1150008AD15000899150008B5
:103BE00085150008D515000800000000D91600084A
:103BF000C516000801170008ED160008F9160008A0
:103C0000E5160008D1160008BD1600085D1700086B
:103C100000000000010000000000000002000000A1
:103C200000000000051900086D1900084000400060
:103C30004038002050380020020000000000000042
:103C40000300000000000000B1190008000000009F
:103C5000100000006038002000000000010000009B
:103C600000000000043B0020010102004172647565
:103C700050696C6F740025424F415244252D424CCF
:103C8000002553455249414C25000000F52200080B
:103C90005D22000871180008D922000843000000C6
:103CA000A43C000809024300020100C032090400DC
:103CB0000001020201000524001001052401000199
:103CC000042402020524060001070582030800FF00
:103CD00009040100020A000000070501024000007B
:103CE000070581024000000012000000F03C0008BF
:103CF000120110010200004083044057000201023B
:103D0000030100000403090425424F4152442500E9
:103D10004633354C696768746E696E6700303132BE
:103D20003334353637383941424344454600000084
:103D30000040000000400000004000000040000083
:103D4000000001000000020000000200000002006C
:103D5000000002000000020000000200000002005B
:103D600000000000F91A0008D91D0008851E00088F
:103D700040004000643B0020643B00200100000044
:103D8000743B0020800000004001000003000000A0
:103D90006D61696E00000000B03D0008803B0020AE
:103DA000783D0020010000001935000800000000E7
:103DB00069646C6500000000A000A802000000001B
:103DC000AAAAAAAA50001400FFFF00000077000072
:103DD00070A70A000000000000000000AAAAAAAA1A
:103DE00000000000FFFF00000000000000000000D5
:103DF0000000100200000000AAAAAAAA0000000108
:103E0000FFFB000000000000000008002000000090
:103E100000000000AAAAAAAA10000000FFFF0000EC
:103E2000000800000000000000000000000000008A
:103E3000AAAAAAAA00000000FFFF000000000000DC
:103E4000000000000000000000000000AAAAAAAACA
:103E500000000000FFFF0000000000000000000064
:103E60000000000000000000AAAAAAAA00000000AA
:103E7000FFFF000000000000000000000000000044
:103E8000000000000A000000000000000300000025
:103E90000000000000000000000000000000000022
:103EA0000000000000000000000000000000000012
:103EB0000000000000000000FF0096000000000865
:103EC00004000000043D00080000000000000000A5
:103ED00000000000000000000000000000000000E2
:00000001FF
